:020000040000FA
:100000000C945D000C9485000C9485000C94850084
:100010000C9485000C9485000C9485000C9485004C
:100020000C9485000C9485000C9485000C9485003C
:100030000C9485000C9485000C9485000C9485002C
:100040000C94BB020C9485000C9485000C948500E4
:100050000C9485000C9485000C9485000C9485000C
:100060000C9485000C94850000000008000201003B
:100070000003040700000000000000000000000072
:10008000250028002B0000000000240027002A0083
:10009000040404040404040402020202020203032E
:1000A0000303030301020408102040800102040836
:1000B0001020010204081020990411241FBECFEF64
:1000C000D8E0DEBFCDBF11E0A0E0B1E0EAE3FEE0A2
:1000D00002C005900D92AC32B107D9F721E0ACE235
:1000E000B1E001C01D92A335B207E1F710E0CDE504
:1000F000D0E004C02197FE010E941507CC35D1073E
:10010000C9F70E9405030C941B070C94000090E0B3
:10011000FC01EC55FF4F249180579F4FFC018491C7
:10012000882399F090E0880F991FFC01EA57FF4F50
:10013000A591B491FC01E458FF4F859194918FB73C
:10014000F894EC91E22BEC938FBF0895AF92BF929D
:10015000CF92DF92EF92FF920F931F93CF93DF9393
:100160006C017B018B01040F151FEB015E01AE18C2
:10017000BF08C017D10759F06991D601ED91FC91E4
:100180000190F081E02DC6010995892B79F7C50111
:10019000DF91CF911F910F91FF90EF90DF90CF9063
:1001A000BF90AF90089590E0FC01E859FF4F249173
:1001B000FC01EC55FF4F3491FC01E057FF4FE491F7
:1001C000EE23C9F0222339F0233001F1A8F42130C5
:1001D00019F1223029F1F0E0EE0FFF1FE458FF4F34
:1001E000A591B4918FB7F894EC91611126C0309528
:1001F0003E233C938FBF08952730A9F02830C9F0E3
:10020000243049F7809180008F7D03C08091800069
:100210008F7780938000DFCF84B58F7784BDDBCF6D
:1002200084B58F7DFBCF8091B0008F778093B00035
:10023000D2CF8091B0008F7DF9CF3E2BDACF0895D9
:1002400090E080E00895FC0101900020E9F73197EB
:10025000AF01481B590BBC018BE391E00C94A60045
:100260008F929F92AF92BF920F931F93CF93DF9382
:10027000CDB7DEB7A1970FB6F894DEBF0FBECDBFE6
:1002800019A2423008F44AE08E010F5D1F4F842E00
:10029000912CB12CA12CA50194010E94F306E62F0C
:1002A000B901CA01EA30F4F4E05DD801EE938D01A2
:1002B000232B242B252B79F790E080E0109719F061
:1002C000CD010E942301A1960FB6F894DEBF0FBEA8
:1002D000CDBFDF91CF911F910F91BF90AF909F90B5
:1002E0008F900895E95CE1CFCF93DF93EC0160E05C
:1002F0008E810E94D30061E08E810E94D30060E075
:100300008E810E94D3008BE891E00197F1F7DF9195
:10031000CF910895CF92DF92EF92FF920F931F93A8
:10032000CF93DF936C017C0187E0E80EF11CD0E0F5
:10033000C0E0062F10E0B8010C2E02C0759567953D
:100340000A94E2F76170F70181917F010E94D30066
:100350002196C430D10579F7C601DF91CF911F9165
:100360000F91FF90EF90DF90CF900C947401CF929B
:10037000DF92EF92FF920F931F93CF93DF93EC01E5
:10038000F62E642F8C810E94D3008D818F3F19F04F
:1003900060E00E94D3000F2D10E08F8584FF25C000
:1003A0006E0187E0C80ED11CF12CE12CB8010E2C97
:1003B00002C0759567950A94E2F76170F601819124
:1003C0006F010E94D300FFEFEF1AFF0A88E0E816E2
:1003D000F10461F7CE01DF91CF911F910F91FF9052
:1003E000EF90DF90CF900C947401B80184E0759584
:1003F00067958A95E1F7CE010E948A016F2DCE01A3
:10040000DF91CF911F910F91FF90EF90DF90CF90F0
:100410000C948A0140E0682F8BE391E00C94B701C3
:1004200081E00E940A028BE39FE10197F1F70895B2
:10043000CF93DF93823029F490914A019860909392
:100440004A0180934E0110924F0180E48093500145
:1004500080E18093510180E58093520180913F01BA
:100460000E948700809140018F3F11F00E94870019
:10047000809141010E948700CBE3D1E09E012B5384
:10048000314080914A0184FD0AC084E090E02196C9
:10049000281739073CF48E810E948700EFCF88E04F
:1004A00090E0F5CF8BE39DE00197F1F760E080915C
:1004B0003F010E94D30060E0809141010E94D3007F
:1004C000809140018F3F19F060E00E94D30080913D
:1004D0004A0184FD34C063E08BE391E00E948A010D
:1004E000CBE4D6E4CE010197F1F763E08BE391E032
:1004F0000E948A012197F1F763E08BE391E00E946B
:100500008A0183E592E00197F1F762E08BE391E0E5
:100510000E948A0180914A0180620E940A0284E05E
:1005200080934B018CE00E940A020E94100282E03C
:1005300080934C0186E0DF91CF910C940A02806297
:100540000E940A028BE496E40197F1F780914A0138
:1005500080620E940A0283E592E00197F1F78091A0
:100560004A0180620E940A02D5CF41E00E94B70191
:1005700081E090E008951F920F920FB60F92112420
:100580002F933F938F939F93AF93BF9380913101AC
:1005900090913201A0913301B0913401309130013A
:1005A00023E0230F2D3758F50196A11DB11D20938F
:1005B00030018093310190933201A0933301B093C5
:1005C000340180912C0190912D01A0912E01B091C8
:1005D0002F010196A11DB11D80932C0190932D0137
:1005E000A0932E01B0932F01BF91AF919F918F9156
:1005F0003F912F910F900FBE0F901F90189526E8F6
:10060000230F0296A11DB11DD2CF789484B58260CC
:1006100084BD84B5816084BD85B5826085BD85B5A6
:10062000816085BD80916E00816080936E00109224
:10063000810080918100826080938100809181009F
:100640008160809381008091800081608093800030
:100650008091B10084608093B1008091B00081608E
:100660008093B00080917A00846080937A008091BA
:100670007A00826080937A0080917A008160809312
:100680007A0080917A00806880937A001092C1008D
:1006900082E00E94180280E4B82ECBE3DFE100E0A4
:1006A00010E0B0927C0080917A00806480937A00A0
:1006B00080917A0086FDFCCF80917800609179006E
:1006C000762F682F70933A0160933901072E000C42
:1006D000880B990B0E94CC0520E030E040EA50E402
:1006E0000E94810620E030EC4FE754E40E94290587
:1006F00060933501709336018093370190933801F0
:1007000082E00E940A02CE010197F1F78CE091E0AD
:100710000E942301E1E080914E018111E0E0E1952A
:10072000F0E0E55CFE4F8489885F80680E940A02E1
:10073000C0903901D0903A010D2C000CEE08FF0852
:100740004AE0C701B601F7FE0EC041E06DE28BE35F
:1007500091E00E94B70166277727CB016C197D09CC
:100760008E099F094AE00E943001E0914E01E2307B
:1007700008F03FC0E150F0E0E55CFE4F84898068FE
:100780000E940A0285E191E00E942301E0914E015E
:10079000E23088F5E150F0E0E55CFE4F8489875F48
:1007A00080680E940A02C0903501D0903601E09026
:1007B0003701F0903801A7019601C701B6010E94E8
:1007C000EE068823D1F08FE191E00E942301809111
:1007D000390190913A01813E23E0920709F0A1C0CE
:1007E0000E9410020115110509F45BCF0E94000060
:1007F00058CFE1E0C0CFE1E0CECF26013701E89449
:1008000077F82FEF3FEF4FE75FE7C301B2010E9498
:10081000EE0681110DC02FEF3FEF4FE75FE7C301F9
:10082000B2010E94240518161CF483E291E0CDCF9A
:100830002FEF3FEF4FE75FE4C701B6010E947C0650
:1008400018161CF487E291E0C0CF2FEF3FEF4FE77F
:100850005FECC701B6010E94240587FDF3CF20E0BD
:1008600030E0A901C701B6010E94240587FF0AC034
:1008700041E06DE28BE391E00E94B701F7FAF0945A
:10088000F7F8F0942AE037ED43EA5BE3C701B601DD
:100890000E94B8042B013C010E949B056B017C0166
:1008A0000E94CA059B01AC01C301B2010E94B704BA
:1008B0002B013C014AE0C701B6010E94300141E032
:1008C0006EE28BE391E00E94B70120E030E040E26D
:1008D00051E4C301B2010E9481062B013C010E9438
:1008E0009B056B01F12CE12C4AE0C701B6010E9487
:1008F0003001C701B6010E94CA059B01AC01C301CA
:10090000B2010E94B70420E030E040E251E40E94CE
:1009100081060E949B0590E080E04AE00E94300141
:1009200056CF8C35910509F45BCF099709F05ACF62
:1009300057CFEBE3F1E01382128284E091E09183E0
:1009400080838CE084838FEF85838BE086838AE0CD
:10095000878389E0808788E0818787E082871386A4
:10096000148615861686178681E00C941802505856
:10097000BB27AA270E94CF040C9442060E9434068B
:1009800038F00E943B0620F039F49F3F19F426F41A
:100990000C9431060EF4E095E7FB0C942B06E92F3E
:1009A0000E94530658F3BA17620773078407950726
:1009B00020F079F4A6F50C9475060EF4E0950B2E54
:1009C000BA2FA02D0B01B90190010C01CA01A001A1
:1009D0001124FF27591B99F0593F50F4503E68F1FC
:1009E0001A16F040A22F232F342F4427585FF3CF3D
:1009F000469537952795A795F0405395C9F77EF40E
:100A00001F16BA0B620B730B840BBAF09150A1F056
:100A1000FF0FBB1F661F771F881FC2F70EC0BA0FDC
:100A2000621F731F841F48F4879577956795B79564
:100A3000F7959E3F08F0B0CF9395880F08F099275F
:100A4000EE0F9795879508950E94070608F481E0B8
:100A500008950E943D050C9442060E943B0658F002
:100A60000E94340640F029F45F3F29F00C942B06D5
:100A700051110C9476060C9431060E94530668F3CB
:100A80009923B1F3552391F3951B550BBB27AA2747
:100A900062177307840738F09F5F5F4F220F331F81
:100AA000441FAA1FA9F335D00E2E3AF0E0E832D049
:100AB00091505040E695001CCAF72BD0FE2F29D04C
:100AC000660F771F881FBB1F261737074807AB071E
:100AD000B0E809F0BB0B802DBF01FF2793585F4F93
:100AE0003AF09E3F510578F00C942B060C94760654
:100AF0005F3FE4F3983ED4F3869577956795B79575
:100B0000F7959F5FC9F7880F911D9695879597F97F
:100B10000895E1E0660F771F881FBB1F62177307F8
:100B20008407BA0720F0621B730B840BBA0BEE1F0D
:100B300088F7E09508950E945B0688F09F5798F02B
:100B4000B92F9927B751B0F0E1F0660F771F881FD2
:100B5000991F1AF0BA95C9F714C0B13091F00E94EC
:100B60007506B1E008950C947506672F782F8827D5
:100B7000B85F39F0B93FCCF3869577956795B39513
:100B8000D9F73EF490958095709561957F4F8F4F82
:100B90009F4F0895E89409C097FB3EF49095809587
:100BA000709561957F4F8F4F9F4F9923A9F0F92F33
:100BB00096E9BB279395F695879577956795B795B1
:100BC000F111F8CFFAF4BB0F11F460FF1BC06F5F97
:100BD0007F4F8F4F9F4F16C0882311F096E911C0A9
:100BE000772321F09EE8872F762F05C0662371F0CA
:100BF00096E8862F70E060E02AF09A95660F771FDE
:100C0000881FDAF7880F9695879597F90895990FB9
:100C10000008550FAA0BE0E8FEEF16161706E807C6
:100C2000F907C0F012161306E407F50798F0621BE7
:100C3000730B840B950B39F40A2661F0232B242BBC
:100C4000252B21F408950A2609F4A140A6958FEFDB
:100C5000811D811D089597F99F6780E870E060E02D
:100C600008959FEF80EC089500240A941616170645
:100C700018060906089500240A941216130614068D
:100C800005060895092E0394000C11F4882352F0F0
:100C9000BB0F40F4BF2B11F460FF04C06F5F7F4FA8
:100CA0008F4F9F4F089557FD9058440F551F59F08F
:100CB0005F3F71F04795880F97FB991F61F09F3F49
:100CC00079F087950895121613061406551FF2CF72
:100CD0004695F1DF08C0161617061806991FF1CFC2
:100CE00086957105610508940895E894BB276627E9
:100CF0007727CB0197F908950E94070608F48FEF34
:100D000008950E9494060C9442060E94340638F01E
:100D10000E943B0620F0952311F00C942B060C94B6
:100D2000310611240C9476060E94530670F3959FA9
:100D3000C1F3950F50E0551F629FF001729FBB27D2
:100D4000F00DB11D639FAA27F00DB11DAA1F649F6E
:100D50006627B00DA11D661F829F2227B00DA11D21
:100D6000621F739FB00DA11D621F839FA00D611DA7
:100D7000221F749F3327A00D611D231F849F600DC8
:100D8000211D822F762F6A2F11249F5750409AF0F1
:100D9000F1F088234AF0EE0FFF1FBB1F661F771F7D
:100DA000881F91505040A9F79E3F510580F00C9448
:100DB0002B060C9476065F3FE4F3983ED4F38695B9
:100DC00077956795B795F795E7959F5FC1F7FE2BE8
:100DD000880F911D9695879597F908950E940706AB
:100DE000880B990B0895A1E21A2EAA1BBB1BFD01CB
:100DF0000DC0AA1FBB1FEE1FFF1FA217B307E407FA
:100E0000F50720F0A21BB30BE40BF50B661F771F51
:100E1000881F991F1A9469F7609570958095909531
:100E20009B01AC01BD01CF010895EE0FFF1F05909E
:100E3000F491E02D0994F894FFCF00000000B50272
:100E4000A60020011F01416E616C6F673A200054BB
:100E5000656E73696F6E3A20006E616E00696E6632
:060E6000006F7666000041
:107E0000112484B714BE81FFF0D085E080938100F7
:107E100082E08093C00088E18093C10086E0809377
:107E2000C20080E18093C4008EE0C9D0259A86E02C
:107E300020E33CEF91E0309385002093840096BBD3
:107E4000B09BFECF1D9AA8958150A9F7CC24DD24C4
:107E500088248394B5E0AB2EA1E19A2EF3E0BF2EE7
:107E6000A2D0813461F49FD0082FAFD0023811F036
:107E7000013811F484E001C083E08DD089C08234E0
:107E800011F484E103C0853419F485E0A6D080C0E4
:107E9000853579F488D0E82EFF2485D0082F10E0AE
:107EA000102F00270E291F29000F111F8ED06801E7
:107EB0006FC0863521F484E090D080E0DECF843638
:107EC00009F040C070D06FD0082F6DD080E0C81688
:107ED00080E7D80618F4F601B7BEE895C0E0D1E017
:107EE00062D089930C17E1F7F0E0CF16F0E7DF06D8
:107EF00018F0F601B7BEE89568D007B600FCFDCFD4
:107F0000A601A0E0B1E02C9130E011968C91119780
:107F100090E0982F8827822B932B1296FA010C0160
:107F200087BEE89511244E5F5F4FF1E0A038BF0790
:107F300051F7F601A7BEE89507B600FCFDCF97BE46
:107F4000E89526C08437B1F42ED02DD0F82E2BD052
:107F50003CD0F601EF2C8F010F5F1F4F84911BD097
:107F6000EA94F801C1F70894C11CD11CFA94CF0C13
:107F7000D11C0EC0853739F428D08EE10CD085E9AC
:107F80000AD08FE07ACF813511F488E018D01DD067
:107F900080E101D065CF982F8091C00085FFFCCF94
:107FA0009093C60008958091C00087FFFCCF809118
:107FB000C00084FD01C0A8958091C6000895E0E648
:107FC000F0E098E1908380830895EDDF803219F02E
:107FD00088E0F5DFFFCF84E1DECF1F93182FE3DFCA
:107FE0001150E9F7F2DF1F91089580E0E8DFEE27F6
:047FF000FF270994CA
:027FFE00040479
:00000001FF
